:100000009302000273A00231370101006128A94860
:100010007300000082808548730000008280914850
:10002000730000008280AD48730000008280930856
:1000300010087300000082809308500873000000CD
:10004000828093087008730000008280732510C0BE
:100050008280732500C082809308600873000000CE
:1000600082800589F322008093920248B3E2A200C5
:10007000739002808280954873000000828093080C
:100080000008730000008280A14873000000828095
:1000900093083008730000008280930840087300C2
:1000A000000082804EB822F44AF052EC5AE862E432
:1000B0006AE001491304001B130BD004930BE00406
:1000C000130CF004930C0005130D1005930D20057F
:1000D00093093005130A400593043400994A130527
:1000E0001903930510040C88488866AC89371305FA
:1000F0002004088866AC253F13053004088866ACE8
:100100003D3713054004088866AC153713055004C5
:10011000088866AC293F13056004088866AC013F77
:1001200013057004088866AC193713058004088825
:1001300066ACF53D13059004088866ACCD3D13050B
:10014000A004088866ACE5351305B004088866ACE1
:10015000F93D1305C004088866ACD13D2300640155
:1001600066ACF1352300740166ACD13523008401FF
:1001700066AC753D2300940166AC553D2300A40197
:1001800066AC75352300B40166AC553523003401E7
:1001900066AC713D2300440166AC513D0509E31096
:1001A00059F522740279626A426B226C026D4EBE6E
:0A01B00041310030303030303000B3
:00000001FF
